:10000000830100308A003B28E50003088301E400F7
:100010002B088100AA0AAC0A00308A002C081F397C
:10002000142086000B1135288207083409340A345D
:100030000C340D340E340E340F340F340F340E34B0
:100040000E340D340C340A340934083406340534C3
:1000500003340234013401340034003400340134F8
:1000600001340234033405340634831264088300F7
:10007000E50E650E090022308400593051202030F1
:1000800084002230512083010730E300F730E20082
:1000900059308400623055208301442D04068001CC
:1000A000840A0406031D4E280034F00060208000FE
:1000B000840A040870060319003456288312E200EB
:1000C000E31B692863088A006208E20A0319E30A4D
:1000D00082008313631883176208E20A8400000811
:1000E00008008207F6348234A834603484346434DF
:1000F000FA34C234E034E434E634E834E434C2346C
:10010000C634D634CA34E4345A3460345C3462348D
:1001100062345A3462346C34CC346C3464347034A9
:020120000034A9
:1004360083122C232C3A8312031908001C2A8B12D0
:1004460083169B001C141A088B1683120800F000F2
:100456000030711870070310F00D0310F10CF1084D
:10046600031908002C2A452A4830D5003D2A831254
:10047600560888228312D50A55032222D600D608AA
:10048600031D3A2A83120800F401F5010310F30C48
:10049600F20C031C552A7008F40771080318710A38
:1004A600F5070310F00DF10D7208730403190034FB
:1004B600492A3030DA00DB00D50083125A08D90009
:1004C6005B08DA005508DB002C23D5002E3A031909
:1004D600702A55082C3A031D602A83120800303012
:1004E600DD00DE00D50083125D08DC005E08DD005D
:1004F6005508DE002C23D5002E3A0319862A550806
:100506002C3A031D762A831208008511A118851539
:100516008312D8000A30D7005130B000211C972A28
:100526005A30B007B00B952A64008312581CA02AD3
:100536008515A11CA42A8511A42A8511A11CA42A0B
:10054600851503148312D80CD70B8F2A0800D50102
:10055600D601D701D800C32A0A30F200F3015608A3
:10056600F1005508F0004722570858078400000894
:100576000F397407D50075080318750AD600D70A0F
:10058600033083125702031CAF2A5608F1005508A0
:10059600F00008002C23BB002C23BC002C23BD003C
:1005A6002C23BE002C23BF002C23C0002C23C1000B
:1005B6001B222C23C2002C232C23C3002C23C40073
:1005C6002C23C5002C23C6002C23C7002C23C800CF
:1005D6002C23C9002C23CA001B222C23CB008312F8
:1005E600080041308822543088220B30882204309B
:1005F60088227F301E2B2C23D50083169C18012BB6
:100606008312550883169B0083122C2383169A00A7
:1006160003108B1B03148B1383161C1555309D007A
:10062600AA309D009C141C1103188B179C18192BBB
:10063600831255082222882283122C23D500573A8A
:100646000319FE2A83125508523A031D08002C236B
:100656001D2B332B6400061E322B0510342B05147C
:100666008312051A382BA1182D2B051E3C2BA11C15
:100676002D2BD6011E30B000B00B3F2B0830D70013
:10068600640051308312B000211C4D2B5A30B00744
:10069600B00B4B2B03108312D60CA11C552B051A3D
:1006A600582B572B051E582BD617D70B432B5130DB
:1006B600B000211C632B5A30B007B00B602B83129D
:1006C600560808006400D701D80008305702831284
:1006D60003180800A0135818A0170310201F882B12
:1006E600A80CA90CA01F792B01307A2B0030F00042
:1006F600031C7F2B0130802B0030F0060319872B5B
:100706008430A8060830A90603108312D80C211ECF
:10071600912B20302A020318952B8C2B3A302A0273
:10072600031C912BAA01A01FAB2BAE0AA11DB42B53
:100736002E08053A031DB42B211EA62B20302A02B3
:100746000318AA2BA12B3A302A02031CA62BAA01B6
:10075600211AAF2BC930B02BE630AB001030A10602
:10076600AE01D70A08305702031808006D2B061F82
:1007760005148312D501C62BD601C32B6400D60AF5
:10078600560FC12BD50A550FBF2BD501D50A031914
:10079600DE2B6400061E061FD42BD501D50A0514D0
:1007A600D72B061FD72B0510D6012030560203186B
:1007B600C92BD60AD82B1B302222F000701CE52B41
:1007C6002014E72B831220101B3083122222F00004
:1007D6007019A01CF02B2016F22B83122012831204
:1007E600DF035F0FFA2B16302222DF008312DF08A9
:0A07F600031D082C20302222F00021
:10080000F01B2010213083122222F000F01B201256
:10081000153083122222F000700F112C0330AD002E
:100820001B2C1530831222222D06031D192CAD011D
:100830001B2C8312AD0A8312051521168316811510
:100840008112C930831281008B17FF30A900A800E4
:1008500020131D302222D5008312D5087E300319C3
:10086000342C6523D5032C2C65232017A115AE014C
:10087000D501831255082222D600D50A55080E3A12
:10088000031D462CAD08031D462CD60A83125608BC
:10089000652355080E3A03195C2C392CD50A5503EB
:1008A0002222D6005508153A031D592C2D0B592C20
:1008B000D60A83125608652383125508153A031980
:1008C000652C01302D0203184E2C02302D02031C22
:1008D000722CAE30652392306523883065238A30D0
:1008E000652383122D08023A031D7D2C6430652395
:1008F000403065236330652383122D08033A031DBE
:10090000882C64306523403065236530652383126D
:100910002D08043A031D932C66306523403065236F
:100920006730652383122D08053A031D9D2C68301E
:1009300065234030652369306523033083126523C6
:10094000F0306523211DBB2C3E306523D5010030DE
:100950008A0083125508712000380319302D0030A9
:100960008A008312D50A55037120F0000310700C21
:1009700083126523A72C213083126523D50108300B
:1009800055020318CB2C831255083B3E8400000807
:100990006523D50ABF2C1E30831222226523D50180
:1009A000093055020318DC2C83125508433E84009D
:1009B00000086523D50AD02C1F308312222265231C
:1009C000201C022DD501033055020318EF2C831291
:1009D0005508593E840000086523D50AE32C2F30C2
:1009E00083126523D501033055020318022D8312AB
:1009F00055085C3E840000086523D50A0330550283
:100A0000031CF72C8312201E1D2D2F30652341302F
:100A100065233D3065232708303E65232608303E98
:100A200065232508303E65232408303E65232308CE
:100A3000303E65232208303E652320308312D500E6
:100A4000262D831256087F3965238312D50A550354
:100A50002222D600D6080319302DDF080319212DD4
:100A600083122013FF30A906A80629086523280849
:100A70006523A1117E3065237E30652305118B131C
:100A8000061F0510831208000830D300D40164004B
:100A90008B018B1607309F0083168113F030860080
:100AA0001030850083120510851405110530D10022
:100AB000D2012114A114D001D00A6400831252087B
:100AC0005104031D792D2115BA2321115308D1009A
:100AD0005408D2000310D30DD40D0730540209304E
:100AE00003195302031C782D0830D3000730D400BB
:100AF0008312CF0F812D0230A106A11C812D013060
:100B0000A1062C23CC00243A03198C2D4C08213A41
:100B1000031D5D2DF4225D2D83122C23473A031D06
:100B20005D2D83122C23503A031D5D2D8312861AEE
:100B30009A2DA016CF01D0080319A02D36228312BA
:100B4000D0012C23CC00563A03192019B02D2C23A8
:100B5000543A031D5D2D2C23473A0319652F5D2D53
:100B600083124C08473A031DBE2D2C23473A031D20
:100B70005D2D2C23413A0319C72E5D2D4C08523AA6
:100B8000031D5D2D2C234D3A031D5D2D2C23433A6F
:100B9000031D5D2D83122015023085062C23D108FC
:100BA0000319D203D103B90A0319BA0A1B222C2351
:100BB000563A0319E12E831285142C23CD222C23BF
:100BC00072221B225C221C3083122222003803195D
:100BD000FB2D3C30F200F3011C302222F000F10129
:100BE000472275083A02031DF72D74083902031CC9
:100BF000BF2EA016BF2E5C308312AA227008B70049
:100C00007108B8005930AA227008B5007108B60002
:100C100019302222F000F1017108803AF200380800
:100C2000803A7202031D162E37087002031C282E0C
:100C30003C308312F200F30118302222F000F1015F
:100C400047227408B3007508B400B101B2019B2EAD
:100C500014308312AF001A302222F000F101710823
:100C6000803AF2003808803A7202031D392E3708A4
:100C700070020318412E173083122222B300B401F0
:100C8000632E1A3083122222F200F301173022223F
:100C9000F000F10147227408F0007508F1003808EF
:100CA000F3003708F20072277408B3007508B40027
:100CB0003808F3003708F200FA30F0000030F10194
:100CC00072277408AF07513083122F02031C6A2E5B
:100CD0005030AF00600A0319610A031D732E3508F6
:100CE000E0003608E10060083502B1006108031C2D
:100CF000610A3602B200B21F852E35086002B100CB
:100D00003608031C360A6102B2003208803AF0004D
:100D100080307002B53003193102031C9C2E6830FC
:100D2000F0000130F10031087002B1003208031CFC
:100D3000320A7102B20083122F08F000F10171082B
:100D4000803AF2003208803A7202031DA92E31085F
:100D500070020318B22E00303A020630031939022D
:100D60000318BA2E3A083402031DB82E390833028C
:100D70000318C02EA0163508E0003608E1008312E3
:100D8000A01E5D2DBA23A012B901BA015D2D8312F8
:100D9000A014023085062C232019D52ED108031962
:100DA000D203D103B90A0319BA0A83121B22CD2236
:100DB0002C232C23303A0319E12E3B082C3A031D37
:100DC000E32E85105D2D831285142C231B221B22FC
:100DD000A201A301A401A501A601A7012C23CD0016
:100DE000CC012D3A0319E32D83122608A70025080C
:100DF000A6002408A5002308A4002208A30021308F
:100E0000F1004D08D03E2A22CE00643083124E02FB
:100E1000031C2A2F9C30CE07A30A0A302302031C8E
:100E2000052FF630A307A40A0A302402031C052F5D
:100E3000F630A407A50A0A302502031C052FF63058
:100E4000A507A60A0A302602031C282FF630A6079B
:100E5000A70A052F0A30F1004E0887274C07A20089
:100E60000A302202031C532FF630A207A30A0A30CD
:100E70002302031C532FF630A307A40A0A302402CE
:100E8000031C532FF630A407A50A0A302502031CC1
:100E9000532FF630A507A60A0A302602031C532F4B
:100EA000F630A607A70A83124E08CC000A304C027F
:100EB000031C5D2FF630CC07562F2C23CD002C3A87
:100EC0000319E32D4D082E3AF22E8312A0152C2380
:100ED0005C2283122C234D3A8312031D6A2F2C238C
:100EE0007222E32DF601F11F7C2FF009F00A03199D
:100EF000F103F1097617F61773088039F606F31F28
:100F0000BE2FF209F20A0319F303F309BE2FF00012
:100F1000F4010310FD307107031CAE2FF301F03014
:100F20007105031D962F0430F300F10EF20103103A
:100F3000F30AF10D031C982FF10C710870020318CD
:100F4000F000F20DF30B9C2FF41FA82FF209F20A08
:100F50007208F41F0800F009F00A0800F10C0318E9
:100F6000B72FF10C031CF0010310F00C031C03104D
:100F70007008F200F001F00DA42FF601F401F50164
:100F800072087304031DC72FF001F10100341F30F4
:100F9000F6040310F60AF20DF30D031CCA2FF30C2E
:100FA000F20C73087102031DD72F72087002031C24
:100FB000DF2F7208F0027308031C730AF102F40DAC
:100FC000F50DF60BF61ACF2FF61FEB2FF409F40AE6
:100FD0000319F503F5097408F2007508F300761F8C
:100FE0000034F009F00A0319F103F1090034303438
:100FF000303430343034303430340134FF34FF3462
:02400E00663F0B
:104200008200A0008A00A400B000A20060009C0010
:104210009E0086008200980098006000A4008A003A
:1042200098008200B20040006000030002005A00C3
:10423000140003003200010000003C002F003E008B
:10424000000000000000000000000000000000006E
:10425000000000000000000000000000000000005E
:10426000000000000000000000000000000000004E
:10427000000000000000000000000000000000003E
:10428000000000000000000000000000000000002E
:10429000000000000000000000000000000000001E
:1042A000000000000000000000000000000000000E
:1042B00000000000000000000000000000000000FE
:1042C00000000000000000000000000000000000EE
:1042D00000000000000000000000000000000000DE
:1042E00000000000000000000000000000000000CE
:1042F00000000000000000000000000000000000BE
:00000001FF
